:100000000C940B030C944F030C944F030C944F036C
:100010000C944F030C944F030C944F030C944F0318
:100020000C944F030C944F030C940E0D0C94E00DA4
:100030000C944F030C944F030C944F030C944F03F8
:100040000C944F030C94AA220C944F030C944F036E
:100050000C944F030C94391C0C944F030C944F03D5
:100060000C944F030C944F030C944F030C944F03C8
:100070000C944F030C944F030C944F030C944F03B8
:100080000C944F030C944F030C944F030C944F03A8
:100090000C944F030C944F030C944F030C944F0398
:1000A0000C944F030C944F030C944F034D0E6F0EA2
:1000B0005D0F6F0E5D0FB40ED70E5D0F2C0F3F0F4F
:1000C0002B122B1268126812AB12E91202150215DC
:1000D0000213021503140314D61402150215ED14AD
:1000E00029002B000354E100358100001E000E00A2
:1000F0000B001B7164004D001F003700040014004A
:10010000E1044C00200012000800340050002A00D6
:10011000210036000C002F004F004A0022001D0075
:100120001800330000000254E000E3000000E20089
:1001300000002E77E400E7000000E60000002E7FBC
:1001400023001900070005000000045424000A00E1
:100150001700130052004B002500060015001A007E
:1001600051002C0026000F0011001000E1082800AB
:1001700027002D0016000D7130004E0038001C00C5
:100180000982E50031810000010001000100010049
:10019000010000003A0035003100010001000100BB
:1001A0003B0035022102640001004C003C001E02AD
:1001B00024062202010001003D002D022402240435
:1001C000010001003E0001003700110400000100A1
:1001D0000100010000000100000001000100010019
:1001E00000000100000001003F0024062402230259
:1001F000000001004000220425023500010001003A
:100200004100230426023502370001004200240485
:1002100025041F021E0201004300310026043102A2
:10022000010001004400450001002D020100000012
:1002300001000100010001000100000001000100B7
:100240000100FB000100010001000100F200F900C3
:10025000010001000100F000F100FA00F4000100CB
:1002600001000100F300FC00F500010001000100A5
:100270000100F60000000100010001000000010083
:100280000000010001000100000001000000010069
:100290000100010001000100000001000100010057
:1002A0000100A800A9000100010001000100AC004C
:1002B000AA00B600010001000100AB0050000100DF
:1002C000010001000100520051000100AE000100D8
:1002D000010001004F00000029002B000100E10097
:1002E000358100001E00140004001D7164004D00E3
:1002F0001F001A0016001B00E1044C00200008003B
:100300000700060050002A0021001500090019000E
:100310004F004A00220017000A00050000000100FB
:100320001908E3000000E20000002E770608E7004D
:100330000000E60000002E7F23001C000B001100CF
:1003400000000100240018000D00100052004B00B6
:1003500025000C000E00360051002C002600120073
:100360000F003700E1082800270013003300387120
:1003700030004E002D002F003482E5003181000056
:100380000100010001000100010000000100010066
:100390000100010001000100010001005000010006
:1003A00001000100010052005100010001000100A4
:1003B000010001004F0001000100010001000100E7
:1003C0000100010000000100010001000000010027
:1003D0000000010001000100000001000000010018
:1003E0003F005200510023020000010040002400A1
:1003F00021001E00270001004100250022001F00EF
:1004000037000100420026002300200027000100E1
:1004100043003002300024022E0001004400450059
:100420000100010001000000160345007200670092
:100430006F0044006F007800200045005A00000063
:1004400016034500720067006F0044006F007800DB
:10045000200045005A0000000403090409026D0051
:10046000040100A0FA0904000001030101000921B0
:1004700011010001223F000705810308000A090459
:1004800001000103010200092111010001224D00B8
:100490000705820308000A090402000103000000A6
:1004A0000921110100012236000705830308000A13
:1004B00009040300010300000009211101000122C9
:1004C000390007058403100001120110010000002B
:1004D00008EDFE071301000102000105010906A154
:1004E00001050719E029E715002501950875018127
:1004F00002050819012905950575019102950175F7
:1005000003910105071900297715002501957875D4
:10051000018102C005010980A101850216010026A2
:10052000B7001A01002AB700751095018100C005B7
:100530000C0901A1018503160100269C021A010085
:100540002A9C02751095018100C005010902A101D4
:100550000901A100050919012905150025019505C5
:100560007501810295017503810105010930093189
:100570001581257F95027508810609381581257F2B
:10058000950175088106050C0A38021581257F95AD
:100590000175088106C0C005010906A101050719FA
:1005A000E029E7150025019508750181029501757F
:1005B0000881010508190129059505750191029524
:1005C00001750391010507190029FF150025FF9505
:1005D0000675088100C00000000000000000000057
:1005E00000010204060A0F17202C3A4A5D71879D0C
:1005F000B3C7DAE9F5FCFFFCF5E9DAC7B39D87710B
:100600005D4A3A2C20170F0A060402010000000080
:1006100000000000000011241FBECFEFDAE0DEBFB3
:10062000CDBF04B603FE24C08091EE019091EF018E
:10063000A091F001B091F1018730904BA740B04BF1
:10064000B9F41092EE011092EF011092F0011092A5
:10065000F10114BE84B7877F84BF88E10FB6F89498
:1006600080936000109260000FBEE0E0FFE3099508
:1006700011E0A0E0B1E0E8EDF8E402C005900D92D1
:10068000A433B107D9F711E0A4E3B1E001C01D9292
:10069000AE3EB107E1F70E94520A0C946A240C9412
:1006A000000061110BC0FC018281882321F085EEDE
:1006B0000E94BF1003C085EE0E94871180E090E089
:1006C000089508956091B1017091B2018091B301D4
:1006D0009091B4010E94651B56985E9825982D98BC
:1006E00026982E9827982F9808950C946203569870
:1006F0005E9825982D9826982E9827982F988FEFFA
:1007000090E0909389008093880090938B00809371
:100710008A0090938D0080938C00259A2D9A2FEF5C
:1007200080E792E0215080409040E1F700C0000057
:10073000269A2E9A2FEF80E792E021508040904039
:10074000E1F700C00000279A2F9A2FEF80E792E090
:10075000215080409040E1F700C0000025982D987E
:100760002FEF80E792E0215080409040E1F700C0F9
:10077000000026982E982FEF80E792E021508040CD
:100780009040E1F700C0000027982F9856985E9897
:1007900025982D9826982E9827982F98089589EABD
:1007A0008093800089E08093810024982C983F9862
:1007B0008AB18F748AB96E98479A8BB1806B8BB966
:1007C000769A0E9477030C94610380E28093000183
:1007D0008091340181110EC00E94340481E0809325
:1007E00034012FEF83ED90E3215080409040E1F7FA
:1007F00000C0000080E40E943A048093000181114F
:100800002EC00E94640480930001811128C00E94C0
:10081000640480930001811122C08FE30E9464046C
:100820008093000181111BC00E945C0480E40E943F
:100830003A0480930001811112C08CE00E9464048C
:100840008093000181110BC00E9464048093000119
:10085000811105C08FE30E946404809300010E940F
:100860005C048091000108951092B9008AE08093A1
:10087000B800089594EA9093BC009091BC0097FF53
:10088000FCCF9091B900987F983021F0903111F011
:1008900081E008958093BB0084E88093BC00809140
:1008A000BC0087FFFCCF8091B900887F883111F0B0
:1008B000803471F780E0089584E98093BC008091D2
:1008C000BC0084FDFCCF08958093BB0084E8809336
:1008D000BC008091BC0087FFFCCF9091B900987F4D
:1008E00081E0983209F480E0089584E88093BC00A8
:1008F0008091BC0087FFFCCF8091BB000895809160
:100900000001811115C080E40E943A048093000127
:1009100081110CC082E10E94640480930001811166
:1009200005C08FEF0E946404809300010E945C0464
:1009300084B1807F84B985B1807F85B98AB1837F96
:100940008AB98BB1837F8BB93E98469808950E94EF
:10095000E503809300010E947F0480B38C7080BB0C
:1009600081B3836F81BBA6E3B1E0E4E4F1E08EE004
:100970008E0F11921D928E13FCCF0C94CF03BF9259
:10098000CF92DF92EF92FF920F931F93CF93DF935B
:1009900080910001882379F0809135018F5F8093E9
:1009A0003501811108C00E94E50380930001811187
:1009B00002C00E94770306E311E0C0E0D0E0DD242E
:1009C000D39482E0C82EEE24E394F12CC730D105F5
:1009D00000F580910001811164C080E40E943A0416
:1009E00080930001811112C082E10E94640480930F
:1009F000000181110BC0C7010C2E01C0880F0A94A1
:100A0000EAF780950E946404809300010E945C04D0
:100A100048C0CA30A1F028F4C83059F0C93061F09C
:100A200005C0CC3089F070F0CD3089F0209A28983C
:100A300010C0219A29980DC0229A2A980AC0239A98
:100A40002B9807C0529A01C0539A5B9802C03E9AF5
:100A5000469890EA9A95F1F79FB1799902C082E0A1
:100A600001C080E091709D25982B7C9902C084E0A4
:100A700001C080E0892B7D9902C038E001C030E0E0
:100A8000832B7E9902C020E101C020E0822B9FB120
:100A90009095991F9927991F9295990F907E892B70
:100AA0000FC080910001811149C080E40E943A0486
:100AB00080930001882379F1B12C0E945C048B2D76
:100AC000F8019081981719F08083C09201010E946B
:100AD0007F0421960F5F1F4FCE30D10509F076CFEE
:100AE00080910101882361F1815080930101882365
:100AF00039F08FE99FE00197F1F700C0000020C0B6
:100B0000A4E4B1E0E6E3F1E0CF01825F91919D932F
:100B10008E13FCCF15C083E10E9464048093000112
:100B20008111CACF81E40E943A04809300018111AF
:100B3000C3CF0E947504B82EB094BFCF80E0C0CF61
:100B40000E94750381E0DF91CF911F910F91FF907B
:100B5000EF90DF90CF90BF900895E82FF0E0EC5B2E
:100B6000FE4F808108950895089596E0799FF001E1
:100B7000112494E5899FE00DF11D1124E60FF11D6C
:100B8000EE0FFF1FE052FF4F859194910895880F5B
:100B9000991FFC01E05AF040859194910895880FC7
:100BA000991FFC01E052FF4F8591949108950F9396
:100BB0001F93CF93DF93EC018115904350F5C1153E
:100BC00080E2D80708F0B3C0CB3BD10590F4C83A17
:100BD000D10508F05AC0C53AD10508F04BC0C43061
:100BE000D10508F0BBC1219709F0B5C101E010E0C3
:100BF000F5C1CF3FD10511F008F0B0C1C03FD1051C
:100C000008F092C0CE01805E9109089708F4A6C151
:100C1000A2C1C11591E5D907A8F4C23020E5D207D9
:100C200008F09EC0C11580E5D80709F485C008F01A
:100C300091C0C11520E4D20708F08DC1DD278E01D7
:100C4000106CCCC1C11580E8D80758F4C11590E7E5
:100C5000D90708F07CC1C11520E6D20708F422C1EB
:100C60007AC1C11580E9D80708F075C1DF708E011F
:100C7000106AB4C1C53AD10509F472C1C63AD105AA
:100C800009F071C102E810E4A9C1C83AD10509F41C
:100C90006DC1C93AD10509F46CC1CA3AD10509F44C
:100CA0006BC1CB3AD10509F46AC1CC3AD10509F43C
:100CB00069C1CD3AD10509F468C1C03BD10509F439
:100CC00067C1CE3AD10509F466C1CF3AD10509F41E
:100CD00065C1C13BD10509F464C1C23BD10509F42A
:100CE00063C1C33BD10509F462C1C43BD10509F41A
:100CF00061C1C53BD10509F460C1C63BD10509F40A
:100D00005FC1C73BD10509F45EC1C83BD10509F4F9
:100D10005DC1C93BD10509F45CC1CA3BD10509F4E9
:100D20005BC100E014E45AC18E01106557C1CE01C9
:100D30009F700E94CF0553C10E9426159FEF24E3A8
:100D40008CE0915020408040E1F700C000000E94FC
:100D50005E1C44C18091CD0181608093CD013EC174
:100D60000E94071E811102C00E94ED1D0E94241ED8
:100D700090E09093EE018093ED01C23090E5D907A9
:100D800021F48091ED01816086C0C43020E5D20756
:100D900021F48091ED0182607EC0C63080E5D807E5
:100DA00021F48091ED01846076C0C83090E5D907C8
:100DB00019F48091ED0127C0CA3020E5D20721F453
:100DC0008091ED01806167C0CC3080E5D80721F4C7
:100DD0008091ED0180625FC0CE3090E5D90721F4AB
:100DE0008091ED01806457C0C03120E5D20721F425
:100DF0008091ED0180684FC0C23180E5D80729F4A9
:100E00008091ED018460886046C0C33090E5D907C9
:100E100021F48091ED018E7F3EC0C53020E5D207E0
:100E200021F48091ED018D7F36C0C73080E5D80771
:100E300021F48091ED018B7F2EC0C93090E5D90758
:100E400019F48091ED0126C0CB3020E5D20721F4C2
:100E50008091ED018F7E1FC0CD3080E5D80721F451
:100E60008091ED018F7D17C0CF3090E5D90721F437
:100E70008091ED018F7B0FC0C13120E5D20721F4B5
:100E80008091ED018F7707C0C331D04531F4809157
:100E9000ED018B7F877F8093ED018091ED010E94B2
:100EA000281E9CC08D2F99278F709927813091051E
:100EB000D9F49E012370332702C0880F991F2A9509
:100EC000E2F79C688E0144E0000F111F4A95E1F79C
:100ED00000271370802B912B53E0CC0FDD1F5A9508
:100EE000E1F7C076DD272FC08230910531F4DC2F89
:100EF000CC278E01016F106A71C08330910569F4AF
:100F0000CE018370992701E010E002C0000F111F8D
:100F10008A95E2F7C8019C680FC0049709F05EC08B
:100F2000CE018370992701E010E002C0000F111F6D
:100F30008A95E2F7C8019A6823E0CC0FDD1F2A9555
:100F4000E1F7C07ED7708C010C2B1D2B47C0DF70E2
:100F50008E01106243C000E010E040C08E013EC030
:100F600001E810E43BC003E810E438C002EE14E4EA
:100F700035C009EE14E432C00AEE14E42FC005EBCC
:100F800014E42CC006EB14E429C007EB14E426C0DB
:100F90000CEC14E423C00DEC14E420C003E815E4C9
:100FA0001DC00AE815E41AC002E915E417C004E9F7
:100FB00015E414C001E216E411C003E216E40EC009
:100FC00004E216E40BC005E216E408C006E216E4EB
:100FD00005C007E216E402C00AE216E4C801DF9188
:100FE000CF911F910F91089596E0799FF001112400
:100FF00094E5899FE00DF11D1124E60FF11DEE0F20
:10100000FF1FE052FF4F85919491803E9105E0F4DF
:10101000803C910558F58133910509F46FC048F47F
:101020008932910509F463C08A32910509F46DC0D3
:1010300072C089339105E9F082389105D1F085338A
:10104000910509F44DC067C0833E910581F138F4E4
:10105000803E9105B9F0823E9105D9F05CC0863E94
:10106000910561F1873E9105A1F155C00E94C70528
:1010700008952091ED0120FD02C021FF4CC080EEBB
:1010800090E049C08091ED0180FFF9CF89E390E0C5
:1010900042C08091ED0182FF0EC08091ED0184FF7E
:1010A00003C080E090E037C083EE90E034C08091D0
:1010B000ED0182FFF2CF82EE90E02DC08091ED0134
:1010C00083FF0BC08091ED0184FDEBCF87EE90E0B4
:1010D00022C08091ED0183FFF5CF86EE90E01BC02A
:1010E0008091ED0185FF07C089E290E014C08091F6
:1010F000ED0185FFF9CF85E390E00DC08091ED0112
:1011000086FF07C08AE290E006C08091ED0186FF6D
:10111000F9CF81E390E00E94D705089508950C94DB
:101120008E08809162010895CF93DF9300D01F92C3
:10113000CDB7DEB79C018091E401843019F593E0CE
:1011400099833B832A839093E9008FEF9091E80085
:10115000815095FD06C095ED9A95F1F7000081113B
:10116000F5CF8091E80085FF0DC040E050E063E0DE
:1011700070E0CE0101960E94FE0A8091E8008E7711
:101180008093E8000F900F900F90DF91CF9108951A
:10119000CF93DF9300D01F92CDB7DEB72091E4014B
:1011A000243021F522E029839B838A8383E0809386
:1011B000E9008FEF9091E800815095FD06C095ED14
:1011C0009A95F1F700008111F5CF8091E80085FF35
:1011D0000DC040E050E063E070E0CE0101960E9457
:1011E000FE0A8091E8008E778093E8000F900F90C0
:1011F0000F90DF91CF9108952091E4012430F1F414
:1012000022E02093E9002FEF3091E800215035FDD6
:1012100006C035ED3A95F1F700002111F5CF209188
:10122000E80025FF0BC040E050E065E070E00E9460
:10123000FE0A8091E8008E778093E8000895CF93AE
:10124000DF93EC019091E401943009F046C0809165
:101250000C018823D9F080910D018823B9F0909377
:10126000E9008FEF9091E800815095FD06C095E16F
:101270009A95F1F700008111F5CF8091E80085FF84
:101280002CC040E050E060E170E017C081E0809346
:10129000E9008FEF9091E800815095FD06C095ED33
:1012A0009A95F1F700008111F5CF8091E80085FF54
:1012B00014C040E050E068E070E0CE010E94FE0AF9
:1012C0008091E8008E778093E80080E1FE01A2E53E
:1012D000B1E001900D928A95E1F7DF91CF910895E9
:1012E0008091E301811109C00E94930C0E94F00CCF
:1012F0008091E20084608093E20008951092E301FF
:10130000089508950C9497220E94F41B0E949D2238
:101310000E94960F0C948F0842E061EC81E00E94DD
:101320000D0C42E061EC82E00E940D0C42E061ECA9
:1013300083E00E940D0C42E161EC84E00C940D0C02
:101340008091E601833009F455C030F4813071F0AA
:10135000823009F48EC008958A3009F47AC08B3047
:1013600009F460C0893009F09CC020C08091E5017B
:10137000813A09F096C08091E800877F8093E80069
:101380008091E9019091EA01892B21F460E182E5E5
:1013900091E003C060E080E090E070E00E94490BC3
:1013A0008091E8008B778093E80008958091E501B3
:1013B000813209F076C08091E9019091EA010097AD
:1013C00019F0039709F06DC08091E800877F809342
:1013D000E8008091E80082FD05C08091E401811160
:1013E000F8CF5FC08091F100809362018091E800A6
:1013F0008B7753C08091E501813A09F052C080910A
:10140000E9019091EA01892B09F04BC08091E80035
:10141000877F8093E8008091E80080FFFCCF809177
:101420000C0136C08091E5018132D9F58091E90146
:101430009091EA01892BA9F58091E800877F80933C
:10144000E8000E94420C8091E70180930C010C940B
:1014500026158091E501813221F58091E800877F92
:101460008093E8000E94420C8091E8018093630120
:1014700008958091E501813AA1F48091E800877F89
:101480008093E8008091E80080FFFCCF80916301A9
:101490008093F1008091E8008E778093E8000C94AF
:1014A000420C089584B7877F84BF88E10FB6F89413
:1014B00080936000109260000FBE90E080E80FB64D
:1014C000F89480936100909361000FBE0E94E50F35
:1014D0000E94930C0E94F00C8091E2008460809343
:1014E000E20078940E94760F0E94E70F82E091E07C
:1014F0000E94910F0E9485228091E401853069F459
:101500000E94B51B8091E2018823B1F30E94E01B89
:10151000882391F30E94E80AEFCF0E94ED0FECCFF1
:10152000292F332723303105C9F064F421303105E8
:1015300081F02230310509F043C08DE690E02CE5C2
:1015400034E042C021323105F1F02232310541F15F
:1015500037C082E190E029EC34E036C09927813031
:10156000910541F08230910541F0892B49F5E8E57C
:10157000F4E005C0E0E4F4E002C0E8E2F4E08491C5
:1015800090E09F0121C06430D8F4E62FF0E0EE0F28
:10159000FF1FEE5DFE4F2081318189E090E014C095
:1015A000643070F470E0FB01EE0FFF1FE65EFE4F4B
:1015B00020813181FB01EA5EFE4F808190E004C012
:1015C00080E090E020E030E0FA013183208308954C
:1015D00080E189BD82E189BD09B400FEFDCF809123
:1015E000D8008F7D8093D8008091E0008260809346
:1015F000E0008091E00081FDFCCF0895CF92DF9262
:10160000EF92FF920F931F93CF93DF93EC018B0127
:101610006A010E94610C811133C0C114D10439F0F8
:10162000F60180819181081B190BC80FD91FE12C8D
:10163000F12C0115110519F18091E80085FD16C006
:101640008091E8008E778093E800C114D10449F0BE
:10165000F60180819181E80EF91EF182E08285E039
:101660000FC00E94610C882321F30AC089918093E6
:10167000F10001501109FFEFEF1AFF0ADACF80E005
:10168000DF91CF911F910F91FF90EF90DF90CF905E
:1016900008952091EB013091EC012617370748F0AF
:1016A0006115710539F42091E8002E772093E80048
:1016B00001C0B90140E061157105A9F12091E40173
:1016C000222309F443C0253009F442C02091E800E8
:1016D00023FD40C02091E80022FD32C02091E800A7
:1016E00020FFE9CF4091F3002091F20030E0342B4D
:1016F000FC01CF016115710559F02830310540F426
:1017000081918093F100615071092F5F3F4FF1CFBC
:1017100041E02830310509F040E02091E8002E77C3
:101720002093E800C8CF4111C9CF0AC08091E401DD
:10173000882361F0853061F08091E80083FD0AC064
:101740008091E80082FFF2CF80E0089582E0089562
:1017500083E0089581E008952091EB013091EC0140
:101760002617370748F06115710539F42091E80014
:101770002E772093E80001C0B901FC0120E061153B
:10178000710591F18091E401882309F440C085300E
:1017900009F43FC08091E80083FD3DC08091E800DE
:1017A00082FD2FC08091E80080FFE9CF2091F300F7
:1017B0008091F20090E0922B6115710559F088300C
:1017C000910540F424912093F10031966150710904
:1017D0000196F2CF21E0089709F020E08091E8001F
:1017E0008E778093E800CBCF2111CCCF0AC08091B7
:1017F000E401882361F0853061F08091E80083FD89
:101800000AC08091E80082FFF2CF80E0089582E074
:10181000089583E0089581E00895982F973058F552
:101820009093E900981739F07091EC002091ED0049
:101830005091F00003C0242F762F50E021FF19C0F3
:101840003091EB003E7F3093EB003091ED003D7F17
:101850003093ED003091EB0031603093EB007093EA
:10186000EC002093ED005093F0002091EE0027FF54
:1018700007C09F5FD3CF8F708093E90081E0089508
:1018800080E008958091E50187FF11C08091E80014
:1018900082FD05C08091E4018111F8CF11C08091D3
:1018A000E8008B770BC08091E401882349F0809198
:1018B000E80080FFF8CF8091E8008E778093E80001
:1018C00008952091E4003091E50095E64091EC0008
:1018D000842F817040FF22C08091E80080FD1CC0F1
:1018E0008091E401882391F0853091F08091EB00A4
:1018F00085FD10C04091E4005091E5004217530768
:1019000029F39A01915011F784E0089582E0089537
:1019100083E0089581E0089580E008954091E80013
:1019200042FFDECF08950E94010D0E94090DE0EEF6
:10193000F0E0808181608083E8EDF0E080818F7746
:10194000808319BCA7EDB0E08C918E7F8C93808151
:101950008F7E80831092E30108950F931F93CF939E
:10196000DF930E94010D0E94090DC8EDD0E088812F
:101970008F77888388818068888388818F7D88833A
:1019800019BC1092E4011092E0011092E201109251
:10199000E10100EE10E0F80180818B7F8083888177
:1019A0008160888342E060E080E00E940D0CE1EEFF
:1019B000F0E080818E7F8083E2EEF0E080818160C4
:1019C0008083808188608083F80180818E7F80831E
:1019D000888180618883DF91CF911F910F91089555
:1019E000E8EDF0E080818F7E8083E7EDF0E080819C
:1019F0008160808384E082BF81E08093E3010C9466
:101A0000AD0CE8EDF0E080818E7F80831092E200E3
:101A100008951092DA001092E10008951F920F923B
:101A20000FB60F9211242F933F934F935F936F93B1
:101A30007F938F939F93AF93BF93EF93FF93809187
:101A4000E10082FF0BC08091E20082FF07C080911D
:101A5000E1008B7F8093E1000E94750F8091DA0096
:101A600080FF1FC08091D80080FF1BC08091DA00EA
:101A70008E7F8093DA008091D90080FF0DC080E1D5
:101A800089BD82E189BD09B400FEFDCF81E080936C
:101A9000E4010E94700905C019BC1092E4010E9483
:101AA0007E098091E10080FF19C08091E20080FFF3
:101AB00015C08091E2008E7F8093E2008091E20069
:101AC00080618093E2008091D80080628093D8008A
:101AD00019BC85E08093E4010E9482098091E100B5
:101AE00084FF30C08091E20084FF2CC080E189BD7A
:101AF00082E189BD09B400FEFDCF8091D8008F7DC1
:101B00008093D8008091E1008F7E8093E1008091E6
:101B1000E2008F7E8093E2008091E20081608093FA
:101B2000E2008091E001882311F084E007C08091F9
:101B3000E30087FD02C081E001C083E08093E401FF
:101B40000E9484098091E10083FF29C08091E20016
:101B500083FF25C08091E100877F8093E10082E0D0
:101B60008093E4011092E0018091E1008E7F8093E8
:101B7000E1008091E2008E7F8093E2008091E2009C
:101B800080618093E20042E060E080E00E940D0C02
:101B90008091F00088608093F0000E948109FF919D
:101BA000EF91BF91AF919F918F917F916F915F91D5
:101BB0004F913F912F910F900FBE0F901F9018954E
:101BC0001F920F920FB60F9211242F933F934F93B2
:101BD0005F936F937F938F939F93AF93BF93CF93B5
:101BE000DF93EF93FF93C091E900CF708091EC00F9
:101BF000D82FD17080FDD0E81092E9008091F000DC
:101C0000877F8093F00078940E94240E1092E90060
:101C10008091F00088608093F000CD2BCF70C0934E
:101C2000E900FF91EF91DF91CF91BF91AF919F912B
:101C30008F917F916F915F914F913F912F910F9075
:101C40000FBE0F901F9018951F93CF93DF93CDB7C2
:101C5000DEB7AA970FB6F894DEBF0FBECDBFE5EE94
:101C6000F1E088E08E0F9091F10091938E13FBCFFD
:101C70000E94A0098091E80083FF1FC18091E501C7
:101C80009091E601492F50E04A30510508F015C106
:101C9000FA01EA5AFF4F0C941F24803881F08238F1
:101CA00009F00BC18091E9018F708093E900809168
:101CB000EB0085FB882780F91092E90006C080912F
:101CC000E1019091E201911182609091E800977F8B
:101CD0009093E8008093F1001092F100C8C0282F83
:101CE0002D7F09F0EAC0882319F0823061F0E5C049
:101CF0008091E701813009F0E0C0933009F080E085
:101D00008093E2012BC08091E701811127C080916F
:101D1000E9018F7009F4D1C08093E9002091EB00B4
:101D200020FF1CC0933021F48091EB00806214C02E
:101D30009091EB0090619093EB0021E030E0A901DD
:101D400002C0440F551F8A95E2F74093EA001092B3
:101D5000EA008091EB0088608093EB001092E9002C
:101D60008091E800877F86C08111A7C01091E701AC
:101D70001F778091E3008078812B8093E30080912E
:101D8000E800877F8093E8000E94420C8091E80081
:101D900080FFFCCF8091E30080688093E300111105
:101DA00002C082E001C083E08093E40186C08058D5
:101DB000823008F082C08091E7019091E8018C3D6B
:101DC00053E0950779F583E08A838AE289834FB7E8
:101DD000F894DE01139620E03EE051E2E32FF0E0BC
:101DE00050935700E49120FF03C0E295EF703F5FEE
:101DF000EF708E2F90E0EA3010F0C79601C0C096C9
:101E00008D939D932F5F243149F74FBF8091E80058
:101E1000877F8093E8006AE270E0CE0101960E941D
:101E2000490B14C0AE014F5F5F4F6091E9010E9402
:101E3000900ABC01892B09F440C09091E800977F7B
:101E40009093E80089819A810E94AC0B8091E80010
:101E50008B778093E80031C0803879F58091E80075
:101E6000877F8093E8008091E0018093F10080916A
:101E7000E8008E778093E8000E94420C1EC081111A
:101E80001CC09091E7019230C0F48091E800877FF8
:101E90008093E8009093E0010E94420C8091E00161
:101EA000811106C08091E30087FD02C081E001C07E
:101EB00084E08093E4010E948C098091E80083FF14
:101EC0000AC08091E800877F8093E8008091EB0052
:101ED00080628093EB00AA960FB6F894DEBF0FBE27
:101EE000CDBFDF91CF911F9108950895CF93809139
:101EF000E4018823A1F0C091E900CF709091EC003B
:101F0000892F817090FD80E8C82B1092E9008091A4
:101F1000E80083FD0E94240ECF70C093E900CF91AA
:101F2000089590936901809368010895E091680194
:101F3000F0916901309721F00190F081E02D099432
:101F400080E00895E0916801F0916901309721F0F7
:101F50000280F381E02D09940895E0916801F091E9
:101F60006901309721F00480F581E02D09940895EE
:101F700020916601309167018217930771F0909369
:101F8000670180936601E0916801F09169013097E3
:101F900021F00680F781E02D0994089520916401D5
:101FA000309165018217930771F0909365018093DA
:101FB0006401E0916801F0916901309721F000849B
:101FC000F185E02D0994089508950C94E40F0E9482
:101FD000FA1B0E94A7040C94C01CCF92DF92EF92D0
:101FE000FF920F931F93CF93DF93CDB7DEB72B975D
:101FF0000FB6F894DEBF0FBECDBF0E94BF048BE6C4
:10200000C82E81E0D82E00E010E0E02E802F0E9444
:10201000AD05F60141916F01F42EF826B1F40F5F82
:102020001F4F0E30110589F78FEF89838A831B823A
:102030000E94031C8160782F9D838C8349815A8183
:102040006B818D810E94901040C09091CD0191FFD5
:1020500004C08B870E94B3058B8520E030E04F2DB4
:1020600050E0922FBA01022E02C0759567950A942E
:10207000E2F760FF24C02E83EF8221E030E06901A7
:1020800002C0CC0CDD1C9A95E2F790E08C219D21DA
:10209000892B09F420E028870E94031C8160782F97
:1020A0009A8789874E815F8168858A850E94901012
:1020B000F801E559FE4F8081C826C08206C02F5F17
:1020C0003F4F2630310569F6AACF0E94A71F109115
:1020D0006A010E94960F1817A1F00E94960F809334
:1020E0006A012B960FB6F894DEBF0FBECDBFDF910D
:1020F000CF911F910F91FF90EF90DF90CF900C94B4
:102100008F082B960FB6F894DEBF0FBECDBFDF91C0
:10211000CF911F910F91FF90EF90DF90CF90089596
:10212000CF93DF93CDB7DEB72B970FB6F894DEBF12
:102130000FBECDBF4F83588769877A878B87DE01B3
:10214000119686E0FD0111928A95E9F785E0FE017E
:10215000379601900D928A95E1F749815A816B81FA
:102160007C818D819E810E94C0172B960FB6F894BA
:10217000DEBF0FBECDBFDF91CF9108950895CF93FD
:10218000882309F4C2C0C82F823859F40E94960FE0
:1021900081FDBBC089E30E94691A0E94361B89E356
:1021A0000CC0833879F40E94960F80FDAEC083E5A1
:1021B0000E94691A0E94361B83E50E94AB1ACF91D8
:1021C0000C94361B843859F40E94960F82FD9DC0F2
:1021D00087E40E94691A0E94361B87E4EECF8CEFD9
:1021E0008C0F813A48F48C2F0E94EA2181118DC016
:1021F0008C2F0E94691AE3CF80E28C0F883048F45C
:10220000C77081E001C0880FCA95EAF70E94EF1AF3
:10221000D6CF8BE58C0F833078F4C53A29F0C63AD7
:1022200031F083E890E005C081E890E002C082E8E8
:1022300090E0CF910C94B80F88E58C0F833108F0B3
:1022400064C0C83A39F1C93A41F1CA3A49F1CB3AC6
:1022500051F1CC3A59F1CD3A61F1C03B69F1CE3A36
:1022600071F1CF3A79F1C13B81F1C23B89F1C33BB6
:1022700091F1C43B99F1C53BA1F1C63BA9F1C73B24
:10228000B1F1C83BB9F1C93BC1F1CA3BC9F180E02A
:1022900090E038C082EE90E035C089EE90E032C028
:1022A0008AEE90E02FC085EB90E02CC086EB90E0AA
:1022B00029C087EB90E026C08CEC90E023C08DEC29
:1022C00090E020C083E891E01DC08AE891E01AC048
:1022D00082E991E017C084E991E014C081E292E0C4
:1022E00011C083E292E00EC084E292E00BC085E26E
:1022F00092E008C086E292E005C087E292E002C068
:102300008AE292E0CF910C94CE0FCF91089588236A
:1023100009F44BC0823859F40E94960F81FF45C0E2
:1023200089E30E94691A0E94361B89E30CC0833836
:1023300071F40E94960F80FF38C083E50E94691AED
:102340000E94361B83E50E94AB1A0C94361B84381E
:1023500059F40E94960F82FF28C087E40E94691AF0
:102360000E94361B87E4EFCF9CEF980F913A58F309
:1023700090E2980F983050F4877091E001C0990F67
:102380008A95EAF7892F0E94F51ADFCF9BE5980F0F
:10239000933020F480E090E00C94B80F885A833199
:1023A00020F480E090E00C94CE0F0895882321F073
:1023B0000E94EF1A0C94361B0895882321F00E9486
:1023C000F51A0C94361B0895BF92CF92DF92EF92CC
:1023D000FF920F931F93CF93DF9300D000D000D0D4
:1023E000CDB7DEB725E0FC01DE01119601900D921C
:1023F0002A95E1F7FC01D080118102812581229587
:102400002F7043815481452B09F4FCC21F3F21F4F6
:10241000FFEFDF1609F4F6C27C012E830E94BE1086
:10242000D9821A8369817A81802F0E94651A182FB8
:10243000B92E0E941A1A0E94E1182E81002319F069
:102440000E940C1B2E81EB2DE295EF70F0E0E05A1C
:10245000FF4F0C941F248B2D807F9B2D9F70F92E96
:10246000882319F0F29480EFF822002389F0FF20EE
:1024700009F475C280E2810F883020F48F2D0E940C
:10248000EF1A03C08F2D0E94FF1A0E94361B67C2ED
:10249000812F0E948711FF2009F4B4C2105E8F2D96
:1024A000183018F40E94F51A02C00E94051B2696E7
:1024B0000FB6F894DEBF0FBECDBFDF91CF911F9155
:1024C0000F91FF90EF90DF90CF90BF900C94361B50
:1024D0003B2D307F8B2D8F70303211F08295807FB5
:1024E000112319F0113021F12CC00023B9F022235F
:1024F00009F4A0C1213009F09DC126960FB6F894C9
:10250000DEBF0FBECDBFDF91CF911F910F91FF9026
:10251000EF90DF90CF90BF900C941F1B222319F0F7
:10252000213009F46FC28E830E94221B8E8196C1D6
:10253000002321F0223008F065C27CC1211162C263
:102540008DC1002321F0222309F474C108C2222383
:1025500009F484C119C22B2D26952695237030E0ED
:102560002115310521F021303105D1F04BC2002376
:1025700021F0812F9B2D937002C080E090E0269681
:102580000FB6F894DEBF0FBECDBFDF91CF911F9184
:102590000F91FF90EF90DF90CF90BF900C94B80F09
:1025A000002321F0812F9B2D937002C080E090E0EA
:1025B00026960FB6F894DEBF0FBECDBFDF91CF9148
:1025C0001F910F91FF90EF90DF90CF90BF900C94F0
:1025D000CE0F812F002319F00E94AF1E02C00E946F
:1025E000171F26960FB6F894DEBF0FBECDBFDF9142
:1025F000CF911F910F91FF90EF90DF90CF90BF9000
:102600000C949C1F8B2D837009F07BC00111FAC1C3
:10261000812F829586958770880F880F912F9F70E4
:10262000C92ED12CE12CF12C082E04C0CC0CDD1CC1
:10263000EE1CFF1C0A94D2F714FF12C04FE050E0CA
:1026400060E070E004C0440F551F661F771F8A9535
:10265000D2F7CB01BA01609570958095909503C033
:1026600060E070E0CB012B2D269526952370422F3C
:1026700050E042305105D9F04330510569F16C29E1
:102680007D298E299F294130510551F126960FB69B
:10269000F894DEBF0FBECDBFDF91CF911F910F9198
:1026A000FF90EF90DF90CF90BF900C9408196C29A9
:1026B0007D298E299F2926960FB6F894DEBF0FBE7E
:1026C000CDBFDF91CF911F910F91FF90EF90DF90E1
:1026D000CF90BF900C9424190E940819C701B6012D
:1026E00026960FB6F894DEBF0FBECDBFDF91CF9117
:1026F0001F910F91FF90EF90DF90CF90BF900C94BF
:10270000EC18002319F08B2D817001C08695882369
:1027100009F478C1812F829586958770880F880F7C
:10272000912F9F70C92ED12CE12CF12C082E04C0C2
:10273000CC0CDD1CEE1CFF1C0A94D2F714FF12C057
:102740004FE050E060E070E004C0440F551F661F8A
:10275000771F8A95D2F7CB01BA0160957095809565
:10276000909503C060E070E0CB012B2D2695269557
:102770002370422F50E042305105D9F043305105CB
:1027800069F16C297D298E299F294130510551F12C
:1027900026960FB6F894DEBF0FBECDBFDF91CF9166
:1027A0001F910F91FF90EF90DF90CF90BF900C940E
:1027B000E2196C297D298E299F2926960FB6F89457
:1027C000DEBF0FBECDBFDF91CF911F910F91FF9064
:1027D000EF90DF90CF90BF900C94FE190E94E21909
:1027E000C701B60126960FB6F894DEBF0FBECDBF67
:1027F000DF91CF911F910F91FF90EF90DF90CF90DD
:10280000BF900C94C619103FD1F118F4103E50F44B
:10281000A1C0123F09F463C008F44CC0133F09F48F
:1028200073C098C01F708B2D8F710023A1F00E9480
:102830005F19812F26960FB6F894DEBF0FBECDBF6D
:10284000DF91CF911F910F91FF90EF90DF90CF908C
:10285000BF900C94D6110E948019812F26960FB636
:10286000F894DEBF0FBECDBFDF91CF911F910F91C6
:10287000FF90EF90DF90CF90BF900C94DD1100237C
:10288000A9F02111BFC08B2D8F7126960FB6F89439
:10289000DEBF0FBECDBFDF91CF911F910F91FF9093
:1028A000EF90DF90CF90BF900C94A519223008F0E4
:1028B000A9C0E9CF0023A9F08B2D8F7126960FB602
:1028C000F894DEBF0FBECDBFDF91CF911F910F9166
:1028D000FF90EF90DF90CF90BF900C945F19002392
:1028E00059F38B2D8F7126960FB6F894DEBF0FBE6D
:1028F000CDBFDF91CF911F910F91FF90EF90DF90AF
:10290000CF90BF900C948019002399F08B2D8F717C
:1029100026960FB6F894DEBF0FBECDBFDF91CF91E4
:102920001F910F91FF90EF90DF90CF90BF900C948C
:102930004A1926960FB6F894DEBF0FBECDBFDF91C1
:10294000CF911F910F91FF90EF90DF90CF90BF90AC
:102950000C9440190023A9F0222309F4ADCF812F54
:1029600026960FB6F894DEBF0FBECDBFDF91CF9194
:102970001F910F91FF90EF90DF90CF90BF900C943C
:10298000BF10222309F4ADCF812F26960FB6F894FD
:10299000DEBF0FBECDBFDF91CF911F910F91FF9092
:1029A000EF90DF90CF90BF900C9487114B2D4F701C
:1029B000612FC7010E94510326960FB6F894DEBF1F
:1029C0000FBECDBFDF91CF911F910F91FF90EF9080
:1029D000DF90CF90BF900C9464184B2D4F70612FF7
:1029E000C70126960FB6F894DEBF0FBECDBFDF91AC
:1029F000CF911F910F91FF90EF90DF90CF90BF90FC
:102A00000C94B40526960FB6F894DEBF0FBECDBF6A
:102A1000DF91CF911F910F91FF90EF90DF90CF90BA
:102A2000BF9008950E940C1B0E941C1B0E94E11A7B
:102A30000E94361B0E944D200E949C1F80E090E067
:102A40000E94B80F80E090E00C94CE0F0E94FC1A18
:102A50000C9412150E945A1A292F22952F7030E0DB
:102A60002C3031054CF42A3031056CF422503109F8
:102A70002230310588F407C02C30310549F02F3061
:102A8000310531F009C0803E48F0803F29F406C08E
:102A900093FB882780F9089580E0089581E00895E8
:102AA000CF93DF9300D000D01F92CDB7DEB70F9049
:102AB0000F900F900F900F90DF91CF910895CF93CB
:102AC000DF9300D000D000D0CDB7DEB726960FB68A
:102AD000F894DEBF0FBECDBFDF91CF9108951F9355
:102AE000CF93DF93C091790116E080917A01C817E6
:102AF00099F0D0E01C9FF0011D9FF00D1124E558C6
:102B0000FE4F4081518162817381848195810E9451
:102B10005F152196C770E9CFDF91CF911F9108957E
:102B20004091AB015091AC016091AD017091AE014B
:102B30008091AF019091B0010C945F158091B0012C
:102B400082958F7009F054C08091AD01882309F4FB
:102B50004FC080917901A0917A016091AB01709191
:102B6000AC014091AE015091AF01B6E08A1709F473
:102B70003FC090E041155105C1F17F3F11F46F3F17
:102B8000A1F1B89FF001B99FF00D1124E558FE4F57
:102B9000218172132AC02081621327C02281211152
:102BA00024C0238134812417350710F421503109C2
:102BB000241B350B283C3105C0F42091B0012F7047
:102BC00020612093B00126E0289FF001299FF00D9D
:102BD0001124E058FE4F80818F70806180838BEAE2
:102BE00091E00E94E4110C946F1501968770BECF9E
:102BF0000895CF92DF92EF92FF920F931F93CF939E
:102C0000DF93CDB7DEB762970FB6F894DEBF0FBE85
:102C1000CDBF8C0185E0F801DE011D9601900D927B
:102C20008A95E1F7D8014C9111965C911197129613
:102C30006C9112971396CD90DC9014973091AB0164
:102C40007091AC018091AE019091AF01009709F4B1
:102C50006BC17F3F19F43F3F09F466C1E090AD01BD
:102C6000EE2009F4C0C02091B001C816D90628F0A2
:102C7000F601E81BF90BCF0104C0809590958C0DEF
:102C80009D1DFF24F394883C910578F0F12C207F62
:102C900009F0C6C07C2DD98AC88A89890E9450153E
:102CA0008BEA91E00E94E411B1C0822F807F09F08D
:102CB00046C0751314C0341312C0611110C02F70B8
:102CC00020612093B0010E9490158BEA91E00E9450
:102CD000E4118091B001D80115968C932EC0CD28B7
:102CE00019F15F3F11F44F3FF9F0F62E61111CC04E
:102CF0008091790120917A0136E0821709F45AC057
:102D000090E0389FF001399FF00D1124E558FE4FF7
:102D10007181571306C07081471303C0728171110E
:102D200003C001968770E9CFF62E662309F418C117
:102D30008091B00181608093B001F12C11C17513B5
:102D400008C0341306C0611104C08091B001D801DD
:102D5000C3C04D875E878D859E856A8B0E942A152C
:102D60006A898823E1F16623D1F12091B001822F95
:102D700082958F7090E0029774F08091AB019091F2
:102D8000AC0198878F831986DB86CA862C87CE0193
:102D900007960E94E41186E0F801ABEAB1E00190E9
:102DA0000D928A95E1F70E949E150E949015FF24CE
:102DB000F394D6C04D875E878D859E850E945A1AF2
:102DC000292F22952F7030E0223031050CF0BCC045
:102DD0009F7009F0B6C0805E883008F4C1C0C80199
:102DE0000E94E411E4CFC816D90608F453C0F601D6
:102DF000E81BF90BCF01883C910508F450C0F12C79
:102E00007C2DD98AC88A89890E945015EBEAF1E0A5
:102E100086E0DF011D928A95E9F70E949015A0C017
:102E2000751314C0341312C0611110C08091B00129
:102E3000F8018583C8010E94E41186E0EBEAF1E025
:102E4000DF011D928A95E9F7FE2C8AC04D875E87C7
:102E50008D859E856A8B0E942A156A89882309F4CC
:102E6000BECF662309F4BBCF2091B001822F82959B
:102E70008F7090E002970CF48ECF8091AB0190910F
:102E8000AC019A8389831B82DD82CC822E83CE01A2
:102E900001967FCF809590958C0D9D1DACCFF62E21
:102EA000662309F49CCF75132EC034132CC02091D7
:102EB000B00120FD1FC0822F82958F70D9F0D801FC
:102EC00015962C9315978F3049F08F5F982F929518
:102ED000907F822F8F70892B15968C93C8010E944A
:102EE000E41186E0F801ABEAB1E001900D928A9519
:102EF000E1F793CF86E0F801ABEAB1E001900D92E3
:102F00008A95E1F72DC04D875E878D859E850E944D
:102F10002A15811140CF8091B00181608093B0016A
:102F2000C8010E94E4111CC0662309F458CF4D87E4
:102F30005E878D859E850E942A15882309F44FCFD0
:102F40002ACF811148CF0CC0243031050CF047CF77
:102F50009F7009F440CFF8019581907F09F03BCF35
:102F60008F2D62960FB6F894DEBF0FBECDBFDF91F6
:102F7000CF911F910F91FF90EF90DF90CF90089528
:102F80001F93CF93DF93CDB7DEB72C970FB6F8948E
:102F9000DEBF0FBECDBF4F83588769877A878B8787
:102FA0009C87CE0107960E94F915882369F08F81CE
:102FB00098852A853B85232BF1F19F3F09F063C05B
:102FC0008F3F09F060C037C086E0FE013796DE0112
:102FD000119601900D928A95E1F76F817885EA85C7
:102FE000FB85309741F17F3F11F46F3F21F1209134
:102FF0007A0130E0C90101968770992740917901E3
:1030000050E08417950709F447C069837A83FD83EC
:10301000EC8396E0929FD001939FB00D1124A558A8
:10302000BE4FFE01319601900D929A95E1F7809383
:103030007A010E946F1516E08091790190917A01D2
:103040008917C1F1189FC001112485589E4F0E9415
:10305000F915882379F1E09179011E9FF00111247F
:10306000E558FE4F40815181628173818481958151
:103070000E945F158091790190E0019687709927F1
:1030800080937901D9CF4F81588569857A858B8561
:103090009C850E945F15CFCF0E94261510927A0161
:1030A00010927901EBEAF1E086E0DF011D928A954A
:1030B000E9F7C1CF2C960FB6F894DEBF0FBECDBF97
:1030C000DF91CF911F910895EF92FF920F931F937D
:1030D000CF93DF938C01892B09F46CC0F12CEE2483
:1030E000E394E8012196F8018491843740F4843018
:1030F00008F051C0813081F0823019F15BC0853712
:1031000009F444C0A8F19CE7980F903708F052C02A
:103110008F770E94871141C00E5F1F4FFE01C4913F
:1031200080E28C0F883048F4C7708E2D01C0880F64
:10313000CA95EAF70E940F1B14C08C2F0E94BF1083
:103140002DC00E5F1F4FFE01C49180E28C0F8830AE
:1031500058F4C7708E2D01C0880FCA95EAF70E94F7
:10316000151B0E94361B1AC08C2F0E94871116C097
:103170000E5F1F4FFE01C491CC2381F08FE99FE0C9
:103180000197F1F700C00000C150F6CF0E5F1F4F4E
:10319000FE01F49003C00E94BF108E018F2D882382
:1031A00009F49FCFEFE9FFE03197F1F700C000008D
:1031B0008150F5CFDF91CF911F910F91FF90EF904C
:1031C000089508956093B5017093B6018093B70197
:1031D0009093B8010C9412150F931F930091B501B1
:1031E0001091B6012091B7013091B801DC01CB01FB
:1031F000802B912BA22BB32B8093B5019093B6011A
:10320000A093B701B093B8011F910F910C941215C0
:103210000F931F930091B5011091B6012091B70152
:103220003091B801DC01CB0180239123A223B32389
:103230008093B5019093B601A093B701B093B80104
:103240001F910F910C9412150F931F930091B501CC
:103250001091B6012091B7013091B801DC01CB018A
:1032600080279127A227B3278093B5019093B601B9
:10327000A093B701B093B8011F910F910C94121550
:103280001092B1011092B2011092B3011092B401E8
:103290000C94121541E050E060E070E004C0440F6F
:1032A000551F661F771F8A95D2F74093B10150933F
:1032B000B2016093B3017093B4010C94121541E014
:1032C00050E060E070E004C0440F551F661F771F98
:1032D0008A95D2F78091B1019091B201A091B3018A
:1032E000B091B401482B592B6A2B7B2B4093B10131
:1032F0005093B2016093B3017093B4010C94121512
:1033000041E050E060E070E004C0440F551F661FCC
:10331000771F8A95D2F7409550956095709580916A
:10332000B1019091B201A091B301B091B4014823D1
:1033300059236A237B234093B1015093B2016093D8
:10334000B3017093B4010C94121541E050E060E0B9
:1033500070E004C0440F551F661F771F8A95D2F78F
:103360008091B1019091B201A091B301B091B401EB
:10337000482759276A277B274093B1015093B20110
:103380006093B3017093B4010C9412150F931F93C3
:103390000091B1011091B2012091B3013091B401BB
:1033A000DC01CB01802B912BA22BB32B8093B1019D
:1033B0009093B201A093B301B093B4011F910F9108
:1033C0000C9412150F931F930091B1011091B2014B
:1033D0002091B3013091B401DC01CB018023912312
:1033E000A223B3238093B1019093B201A093B301C0
:1033F000B093B4011F910F910C9412150F931F936A
:103400000091B1011091B2012091B3013091B4014A
:10341000DC01CB0180279127A227B3278093B1013C
:103420009093B201A093B301B093B4011F910F9197
:103430000C9412150895CF92DF92EF92FF920F93A2
:103440001F93CF93DF938C01C090B501D090B6014C
:10345000E090B701F090B8018091B1019091B20174
:10346000A091B301B091B401C82AD92AEA2AFB2A53
:10347000CFE1D0E0D701C6010C2E04C0B695A795C8
:10348000979587950A94D2F780FF06C0B8018C2FD4
:103490000E94F407019721F4219760F780E001C0B2
:1034A0008C2FDF91CF911F910F91FF90EF90DF90C4
:1034B000CF900895CF93DF93EC010E941B1ABE01B9
:1034C0000E94F407DF91CF910895CB010E945A1A10
:1034D000089590910C01992321F090910D01911183
:1034E00009C020910E0130910F01F90132969FEF32
:1034F00040E01FC0982F9695969596959F3050F571
:10350000E0910E01F0910F01E90FF11D877021E0AC
:1035100030E0A90102C0440F551F8A95E2F7CA01A5
:103520009181892B818308959F3F39F04F5F4E3001
:1035300041F051915813F8CF0DC05111F7CF942F8E
:10354000F5CF9F3F39F0F901E90FF11D97FDFA958D
:1035500082830895089590910C01992321F0909110
:103560000D01911109C020910E0130910F01F90157
:103570003296205F3F4F1FC0982F9695969596954F
:103580009F30F0F4E0910E01F0910F01E90FF11D71
:10359000877021E030E0A90102C0440F551F8A95D1
:1035A000E2F7CA018095918189238183089531963C
:1035B000E217F30729F090819813F9CF1082F7CF23
:1035C000089581E090E0E0910E01F0910F01E80F85
:1035D000F91F1082019680319105A9F70895909105
:1035E000CC01892B8093CC01089580959091CC01DA
:1035F00089238093CC0108951092CC010895909175
:10360000CB01892B8093CB01089580959091CB01BC
:1036100089238093CB0108951092CB010895909156
:10362000CA01892B8093CA01089580959091CA019F
:1036300089238093CA0108951092CA010895809346
:10364000B90108951092B901089580910E019091E9
:103650000F01FC0131969C01205F3F4F80E091916A
:1036600091118F5FE217F307D1F70895E0910E01F2
:10367000F0910F018091CC018083E0910E01F091D7
:103680000F0190818091CB01892B8083E0910E0105
:10369000F0910F0190818091CA01892B80838091E4
:1036A000B901882361F0E0910E01F0910F01908142
:1036B000892B80830E94251B81111092B901809172
:1036C0000E0190910F010C94A20FCF92DF92EF9216
:1036D000FF926C01EE24FF24C114D104E104F10433
:1036E00021F0C701B60120E101C020E0C72ED82E8D
:1036F000E92EFF24C114D104E104F10419F0285F7C
:10370000C701B6016B017C0154E0F694E794D794AD
:10371000C7945A95D1F7C114D104E104F10419F00A
:103720002C5FC701B6016B017C0142E0F694E7947F
:10373000D794C7944A95D1F7C114D104E104F10498
:1037400019F02E5FC701B601DC01CB01B695A79534
:1037500097958795892B8A2B8B2B09F02F5F822FCA
:10376000FF90EF90DF90CF9008958091E401843036
:1037700021F11092CE0120E488E190E00FB6F89498
:10378000A895809360000FBE2093600080E00E94A7
:103790008F0883B7817F846083BF83B7816083BFD5
:1037A0007894889583B78E7F83BF88E10FB6F894AD
:1037B00080936000109260000FBE089508950895F0
:1037C000CF930E94DE1B0E94BF040E94DF1BC0E05B
:1037D0008C2F0E94AD05811104C0CF5FCE30C1F7A0
:1037E00001C081E0CF9108950E9426150E94960F96
:1037F0000C948F0882E084BD93E095BD9AEF97BD4D
:1038000080936E0008952FB7F8948091CF01909126
:10381000D001A091D101B091D2012FBF0895CF92D4
:10382000DF92EF92FF920F931F932FB7F89440917E
:10383000CF015091D0016091D1017091D2012FBF81
:103840006A017B01EE24FF248C0120E030E0C016E9
:10385000D106E206F30610F4415051099A01281BE3
:10386000390BC9011F910F91FF90EF90DF90CF901E
:1038700008951F920F920FB60F9211248F939F936A
:10388000AF93BF938091CF019091D001A091D101CE
:10389000B091D2010196A11DB11D8093CF019093EB
:1038A000D001A093D101B093D201BF91AF919F916C
:1038B0008F910F900FBE0F901F9018950E94930C40
:1038C000F8942FEF87EA91E6215080409040E1F78D
:1038D00000C0000087E090EBDC018093EE01909344
:1038E000EF01A093F001B093F1019CE088E10FB6E5
:1038F000F894A895809360000FBE90936000FFCF6E
:10390000EF92FF920F931F93CF93DF93D82FC0E0D6
:103910008C2F0E94AD0500E010E0E82EF12CC701CD
:10392000002E02C0959587950A94E2F780FD06C0A7
:103930000F5F1F4F0630110591F709C0602F7C2FD4
:1039400080E00E94B505D813F3CF81E004C0CF5FBB
:10395000CE30F1F680E0DF91CF911F910F91FF9073
:10396000EF900895CF93C82F8CE20E94801C88238B
:1039700021F08C2FCF910C94801C80E0CF91089582
:10398000CF930E94071E811102C00E94ED1DC5E663
:10399000C15049F00E94BF048FE39CE90197F1F701
:1039A00000C00000F5CF89E20E94B21C811113C152
:1039B0008AE20E94B21C81110E94ED1D85E00E94E6
:1039C000B21C81110E945E1C0E94121E8093CD01C8
:1039D00087E00E94B21C8823A9F18BE10E94B21CEF
:1039E000882351F08091CD0181FB222720F991E0BD
:1039F000922790FB81F90EC08EE00E94B21C8823B2
:103A000061F08091CD0182FB222720F991E092277D
:103A100090FB82F98093CD0115C080E10E94B21C19
:103A20009091CD01882341F093FB222720F981E07A
:103A3000822780FB93F904C0892F809580FB90F941
:103A40009093CD018091CD010E94161E0E94241EEC
:103A50008093ED0180EE0E94B21C882341F080919A
:103A6000ED01982F909590FB80F98093ED0189E30B
:103A70000E94B21C882359F08091ED0181FB22271E
:103A800020F991E0922790FB81F98093ED0182EE7D
:103A90000E94B21C882359F08091ED0182FB2227FD
:103AA00020F991E0922790FB82F98093ED0186EE58
:103AB0000E94B21C882359F08091ED0183FB2227DC
:103AC00020F991E0922790FB83F98093ED0183EE3A
:103AD0000E94B21C882359F08091ED0184FB2227BB
:103AE00020F991E0922790FB84F98093ED0185E322
:103AF0000E94B21C882359F08091ED0185FB22279A
:103B000020F991E0922790FB85F98093ED0181E304
:103B10000E94B21C882359F08091ED0186FB222778
:103B200020F991E0922790FB86F98093ED0181E1E5
:103B30000E94B21C882359F08091ED0187FB222757
:103B400020F991E0922790FB87F98093ED01809115
:103B5000ED010E94281E8091ED0187FB882780F9E6
:103B600080930D0187E20E94B21CC82F8EE10E9453
:103B7000B21C8111C2608FE10E94B21C8111C4602D
:103B800080E20E94B21C8111C86081E20E94B21CD6
:103B90008111C06182E20E94B21C8111C06283E285
:103BA0000E94B21C8111C06484E20E94B21C88236E
:103BB00011F0C06802C0CC2329F08C2F0E941F1E78
:103BC0006C2F03C00E941B1E682F70E080E090E005
:103BD000CF910C94E218CF9108956DEE7EEF80E0C6
:103BE00090E00E94552460E082E090E00E9447242B
:103BF00060E083E090E00E94472460E084E090E091
:103C00000E94472460E085E090E00C94472480E027
:103C100090E00E94412421E08D3E9E4F09F020E07B
:103C2000822F089582E090E00C943924682F82E07E
:103C300090E00C94472483E090E00C943924682FA2
:103C400083E090E00C94472484E090E00C943924C5
:103C5000682F84E090E00C9447248091D50180FF88
:103C60000BC06091130185E0689FB0011124759528
:103C70006795759567952BC081FF09C06091130109
:103C800085E0689FB00111247595679520C082FF7B
:103C900007C06091130185E0689FB001112417C02F
:103CA0009091D6019923D1F060911201961788F76F
:103CB0002091130185E0289F90011124929FA0017B
:103CC000939F500D112470E0CA010E940B246038AC
:103CD000710540F46115710539F002C065E070E0CE
:103CE000862F08958FE7089581E008958091D5018A
:103CF00080FF08C06091110170E07595679575951A
:103D0000679521C081FF06C06091110170E0759533
:103D1000679519C082FF04C06091110170E010C066
:103D20009091D6019923C1F0609110019617A0F7E8
:103D300080911101899FC001112470E00E940B2421
:103D40006038710528F46115710521F0862F0895FA
:103D50008FE7089581E0089561E070E0F4CF803F3F
:103D600021F40E942D1E819504C0813F29F40E94F8
:103D70002D1E8093D9010895823F21F40E942D1EAB
:103D8000819504C0833F29F40E942D1E8093D801A1
:103D90000895893F19F40E94761E05C08A3F31F4C8
:103DA0000E94761E81958093DA0108958B3F21F45D
:103DB0000E94761E819504C08C3F29F40E94761ED5
:103DC0008093DB010895843F21F48091D7018160C5
:103DD00017C0853F21F48091D701826011C0863FD2
:103DE00021F48091D70184600BC0873F21F480913A
:103DF000D701886005C0883F31F48091D701806188
:103E00008093D70108958D3F21F48091D501816081
:103E10000BC08E3F21F48091D501826005C08F3F99
:103E200029F48091D50184608093D5010895803F65
:103E300039F48091D90187FF6CC01092D90169C013
:103E4000813F29F48091D9011816BCF362C090918A
:103E5000D801823F29F497FF5CC01092D80159C065
:103E6000833F19F41916CCF354C0893F41F4809173
:103E7000DA0118160CF04DC01092DA014AC08A3FE0
:103E800029F48091DA0187FF44C0F6CF8B3F39F4E3
:103E90008091DB0187FF3DC01092DB013AC08C3F6F
:103EA00029F48091DB011816BCF333C0843F21F460
:103EB0008091D7018E7F17C0853F21F48091D70173
:103EC0008D7F11C0863F21F48091D7018B7F0BC07D
:103ED000873F21F48091D701877F05C0883F31F467
:103EE0008091D7018F7E8093D70113C08D3F21F43D
:103EF0008091D5018E7F0BC08E3F21F48091D5013A
:103F00008D7F05C08F3F29F48091D5018B7F8093F1
:103F1000D5018091D80181110EC08091D901811104
:103F20000AC08091DA01811106C08091DB01811104
:103F300002C01092D601089587ED91E00E94AD0F66
:103F40000E94031C9093D4018093D30108951F9382
:103F5000CF93DF938091D3019091D4010E940F1CE5
:103F6000AC019091D601992321F02091140130E009
:103F700006C0209115018AE0289F90011124421764
:103F8000530708F486C08091D801C091D901D0911F
:103F9000DA011091DB01811107C0C11176C0D11186
:103FA00074C0111172C075C09F3F19F09F5F90934C
:103FB000D601181624F40E942D1E8093D8018091FA
:103FC000D80187FF05C00E942D1E81958093D801DE
:103FD0001C1624F40E942D1E8093D9018091D901D2
:103FE00087FF05C00E942D1E81958093D9016091A5
:103FF000D801662339F1C091D901CC2319F1772773
:1040000067FD7095872F972F0E941C2323E333E3CE
:1040100043E35FE30E9480230E94E9226093D8017A
:104020006C2F772767FD7095872F972F0E941C2391
:1040300023E333E343E35FE30E9480230E94E9220A
:104040006093D9011D1624F40E94761E8093DA0134
:104050008091DA0187FF05C00E94761E81958093CA
:10406000DA01111624F40E94761E8093DB01809100
:10407000DB0187FF05C00E94761E81958093DB01DE
:10408000DF91CF911F910C949C1F9F3F09F08ECF21
:1040900096CFDF91CF911F910895E7EDF1E085E094
:1040A000DF011D928A95E9F71092D6011092D50191
:1040B0000895833081F128F4813059F08230D1F0B5
:1040C0000895853009F449C0B8F1863009F456C026
:1040D000089580911501262F30E0280F311D2F3FC4
:1040E000310524F4680F6093150108958FEF8093D4
:1040F0001501089580911401262F30E0280F311DFD
:104100002F3F310524F4680F6093140108958FEF59
:1041100080931401089580911301262F30E0280F19
:10412000311D2F3F310524F4680F6093130108956A
:104130008FEF80931301089580911201262F30E0B4
:10414000280F311D2F3F310524F4680F60931201B1
:1041500008958FEF80931201089580911101262F09
:1041600030E0280F311D2F3F310524F4680F609394
:10417000110108958FEF809311010895809110012E
:10418000262F30E0280F311D2F3F310524F4680F12
:104190006093100108958FEF80931001089583308C
:1041A00011F128F4813049F0823091F00895853082
:1041B00081F120F18630C1F10895809115016817D1
:1041C00020F4861B8093150108951092150108951F
:1041D00080911401681720F4861B809314010895C0
:1041E00010921401089580911301681720F4861B22
:1041F0008093130108951092130108958091120184
:10420000681720F4861B8093120108951092120102
:10421000089580911101681720F4861B8093110185
:10422000089510921101089580911001681720F4EB
:10423000861B8093100108951092100108950F932A
:104240001F938D3109F46BC008F03FC08E3009F424
:104250007FC0C0F4873009F469C068F4863009F083
:10426000B1C08091CD01817F8E7F8093CD0181E0AF
:104270008093DD01A8C0883009F4A2C08B3009F416
:104280009FC0A0C0863109F49BC078F4803109F446
:1042900072C0813109F096C00E94261590910D01DF
:1042A00081E0892780930D018BC0893109F488C092
:1042B0008B3109F087C08091CD0181FB222720F945
:1042C00091E0922790FB81F94CC0853309F470C0CE
:1042D00048F4873209F46CC008F459C0893209F4F3
:1042E00067C070C0833438F48A3308F04EC0883316
:1042F00009F466C067C0833409F45AC0883409F0F1
:1043000061C00E9426150FEF13ED20E3015010400D
:104310002040E1F700C000000E945E1C51C00E94D6
:10432000A3220E94960F0E948F084AC09091CD014F
:10433000892F8095817080FB90F929F096609860B4
:104340009093CD0140C0997F977F9093CD0138C065
:104350008091CD0182FB222720F991E0922790FBEA
:1043600082F98093CD01992359F18091CD0181602B
:104370008093CD0125C08091CD0183FB222720F9B8
:1043800091E0922790FB83F9ECCF895301C08D51C6
:1043900041E050E060E070E08A019B0104C0000F42
:1043A000111F221F331F8A95D2F7C901B80104C01B
:1043B00061E070E080E090E00E94E2180E94261523
:1043C00081E001C080E01F910F91089580E0089581
:1043D00080E00895CF93C82F8091DD01813079F07E
:1043E00018F08230E9F187C0E0910E01F0910F01E1
:1043F0008081813169F0823209F07FC009C0E0918B
:104400000E01F0910F018081813111F0823261F44F
:104410008C2F0E94E621811104C08C2F0E941F2145
:104420001DC081E090E01AC08C2F0E94E82181110C
:1044300014C0C43179F048F4CB3079F0C03109F0C0
:1044400060C082E08093DD0108C0C93219F0C83332
:1044500021F057C01092DD0154C081E0817053C03B
:10446000C93289F118F5C43171F1A8F4C73009F0E7
:1044700046C08AE08093150194E19093140193E083
:10448000909313018093120188E08093110188E2D8
:104490008093100134C0CE51C63088F5EC2FF0E087
:1044A000E65DFE4F80818093DC0129C0CE34E9F0C7
:1044B00020F4CB3421F56AE013C0C13579F0C23560
:1044C000F1F461E00DC08091DC01882319F01092B5
:1044D000DC0115C081E08093DD0115C061E006C0FC
:1044E0008091DC010E9459200AC06AE08091DC01C1
:1044F0000E94CF2004C01092DD0180E004C081E062
:1045000002C080E0ABCFCF910895E1E8F0E0808178
:10451000886080838081816080838FB7F89493E086
:104520009093890090ED909388008FBF0895EFE6F7
:10453000F0E08081826080830895EFE6F0E0808182
:104540008D7F80830895EFE6F0E0908182E08927F7
:10455000808308951F920F920FB60F9211242F930C
:104560003F934F935F936F937F938F939F93AF93FB
:10457000BF93EF93FF938091DE019091DF0101964D
:104580009093DF018093DE01811103C082E00E94DD
:104590008F08E091DF01E695E695F0E0EA52FA4FE8
:1045A000E4918091DE018E1303C080E00E948F08A9
:1045B000FF91EF91BF91AF919F918F917F916F91FB
:1045C0005F914F913F912F910F900FBE0F901F90D1
:1045D000189504D06894B1118DC0089570D088F0FA
:1045E0009F5790F0B92F9927B751A0F0D1F0660FDF
:1045F000771F881F991F1AF0BA95C9F712C0B130FA
:1046000081F077D0B1E0089574C0672F782F8827A4
:10461000B85F39F0B93FCCF3869577956795B39538
:10462000D9F73EF490958095709561957F4F8F4FA7
:104630009F4F0895E89409C097FB3EF490958095AC
:10464000709561957F4F8F4F9F4F9923A9F0F92F58
:1046500096E9BB279395F695879577956795B795D6
:10466000F111F8CFFAF4BB0F11F460FF1BC06F5FBC
:104670007F4F8F4F9F4F16C0882311F096E911C0CE
:10468000772321F09EE8872F762F05C0662371F0EF
:1046900096E8862F70E060E02AF09A95660F771F03
:1046A000881FDAF7880F9695879597F9089557FD33
:1046B0009058440F551F59F05F3F71F04795880F90
:1046C00097FB991F61F09F3F79F087950895121627
:1046D00013061406551FF2CF4695F1DF08C01616D3
:1046E00017061806991FF1CF869571056105089484
:1046F0000895E894BB2766277727CB0197F908959B
:104700000BD078C069D028F06ED018F0952309F04E
:104710005AC05FC01124EECFCADFA0F3959FD1F33A
:10472000950F50E0551F629FF001729FBB27F00D5F
:10473000B11D639FAA27F00DB11DAA1F649F6627B4
:10474000B00DA11D661F829F2227B00DA11D621F03
:10475000739FB00DA11D621F839FA00D611D221FBD
:10476000749F3327A00D611D231F849F600D211DA1
:10477000822F762F6A2F11249F5750408AF0E1F044
:1047800088234AF0EE0FFF1FBB1F661F771F881F8D
:1047900091505040A9F79E3F510570F014C0AACF28
:1047A0005F3FECF3983EDCF3869577956795B79578
:1047B000F795E7959F5FC1F7FE2B880F911D9695A2
:1047C000879597F9089597F99F6780E870E060E012
:1047D00008959FEF80EC089500240A94161617069A
:1047E00018060906089500240A94121613061406E2
:1047F00005060895092E0394000C11F4882352F045
:10480000BB0F40F4BF2B11F460FF04C06F5F7F4FFC
:104810008F4F9F4F089597FB072E16F4009407D0F3
:1048200077FD09D00E94252407FC05D03EF4909521
:1048300081959F4F0895709561957F4F0895EE0F74
:10484000FF1F0590F491E02D0994AA1BBB1B51E1B9
:1048500007C0AA1FBB1FA617B70710F0A61BB70BF0
:10486000881F991F5A95A9F780959095BC01CD0195
:104870000895F999FECF92BD81BDF89A992780B528
:104880000895A8E1B0E042E050E00C945C24262FAB
:10489000F999FECF1FBA92BD81BD20BD0FB6F89425
:1048A000FA9AF99A0FBE019608950E944724272F7D
:1048B0000C944824DC01CB01FC01F999FECF06C021
:1048C000F2BDE1BDF89A319600B40D9241505040CE
:0848D000B8F70895F894FFCF3A
:1048D800200291081F09FC08C80894080101BA01C0
:1048E80028080A03140A3F4D363997054A05140566
:1048F800DB046E048704A004B9040102030405065E
:044908000708090093
:00000001FF
